Archive member included to satisfy reference by file (symbol)

c:/program files (x86)/gnu tools arm embedded/5.2 2015q4/bin/../lib/gcc/arm-none-eabi/5.2.1/armv6-m\libgcc.a(_udivsi3.o)
                              ./emlib/em_msc.o (__aeabi_uidiv)
c:/program files (x86)/gnu tools arm embedded/5.2 2015q4/bin/../lib/gcc/arm-none-eabi/5.2.1/armv6-m\libgcc.a(_dvmd_tls.o)
                              c:/program files (x86)/gnu tools arm embedded/5.2 2015q4/bin/../lib/gcc/arm-none-eabi/5.2.1/armv6-m\libgcc.a(_udivsi3.o) (__aeabi_idiv0)
c:/program files (x86)/gnu tools arm embedded/5.2 2015q4/bin/../lib/gcc/arm-none-eabi/5.2.1/armv6-m\libgcc.a(_clzsi2.o)
                              ./emlib/em_cmu.o (__clzsi2)
c:/program files (x86)/gnu tools arm embedded/5.2 2015q4/bin/../lib/gcc/arm-none-eabi/5.2.1/armv6-m\libgcc.a(_aeabi_uldivmod.o)
                              ./emlib/em_usart.o (__aeabi_uldivmod)
c:/program files (x86)/gnu tools arm embedded/5.2 2015q4/bin/../lib/gcc/arm-none-eabi/5.2.1/armv6-m\libgcc.a(_muldi3.o)
                              ./emlib/em_usart.o (__aeabi_lmul)
c:/program files (x86)/gnu tools arm embedded/5.2 2015q4/bin/../lib/gcc/arm-none-eabi/5.2.1/armv6-m\libgcc.a(_udivmoddi4.o)
                              c:/program files (x86)/gnu tools arm embedded/5.2 2015q4/bin/../lib/gcc/arm-none-eabi/5.2.1/armv6-m\libgcc.a(_aeabi_uldivmod.o) (__udivmoddi4)
c:/program files (x86)/gnu tools arm embedded/5.2 2015q4/bin/../lib/gcc/arm-none-eabi/5.2.1/armv6-m\libgcc.a(_clzdi2.o)
                              c:/program files (x86)/gnu tools arm embedded/5.2 2015q4/bin/../lib/gcc/arm-none-eabi/5.2.1/armv6-m\libgcc.a(_udivmoddi4.o) (__clzdi2)
c:/program files (x86)/gnu tools arm embedded/5.2 2015q4/bin/../lib/gcc/arm-none-eabi/5.2.1/../../../../arm-none-eabi/lib/armv6-m\libc_nano.a(lib_a-exit.o)
                              c:/program files (x86)/gnu tools arm embedded/5.2 2015q4/bin/../lib/gcc/arm-none-eabi/5.2.1/../../../../arm-none-eabi/lib/armv6-m/crt0.o (exit)
c:/program files (x86)/gnu tools arm embedded/5.2 2015q4/bin/../lib/gcc/arm-none-eabi/5.2.1/../../../../arm-none-eabi/lib/armv6-m\libc_nano.a(lib_a-impure.o)
                              c:/program files (x86)/gnu tools arm embedded/5.2 2015q4/bin/../lib/gcc/arm-none-eabi/5.2.1/../../../../arm-none-eabi/lib/armv6-m\libc_nano.a(lib_a-exit.o) (_global_impure_ptr)
c:/program files (x86)/gnu tools arm embedded/5.2 2015q4/bin/../lib/gcc/arm-none-eabi/5.2.1/../../../../arm-none-eabi/lib/armv6-m\libc_nano.a(lib_a-init.o)
                              c:/program files (x86)/gnu tools arm embedded/5.2 2015q4/bin/../lib/gcc/arm-none-eabi/5.2.1/../../../../arm-none-eabi/lib/armv6-m/crt0.o (__libc_init_array)
c:/program files (x86)/gnu tools arm embedded/5.2 2015q4/bin/../lib/gcc/arm-none-eabi/5.2.1/../../../../arm-none-eabi/lib/armv6-m\libc_nano.a(lib_a-memcpy-stub.o)
                              ./src/aes.o (memcpy)
c:/program files (x86)/gnu tools arm embedded/5.2 2015q4/bin/../lib/gcc/arm-none-eabi/5.2.1/../../../../arm-none-eabi/lib/armv6-m\libc_nano.a(lib_a-memset.o)
                              c:/program files (x86)/gnu tools arm embedded/5.2 2015q4/bin/../lib/gcc/arm-none-eabi/5.2.1/../../../../arm-none-eabi/lib/armv6-m/crt0.o (memset)
c:/program files (x86)/gnu tools arm embedded/5.2 2015q4/bin/../lib/gcc/arm-none-eabi/5.2.1/../../../../arm-none-eabi/lib/armv6-m\libnosys.a(_exit.o)
                              c:/program files (x86)/gnu tools arm embedded/5.2 2015q4/bin/../lib/gcc/arm-none-eabi/5.2.1/../../../../arm-none-eabi/lib/armv6-m\libc_nano.a(lib_a-exit.o) (_exit)

Allocating common symbols
Common symbol       size              file

SystemCoreClock     0x4               ./CMSIS/efm32hg/system_efm32hg.o
rawPacket           0x110             ./src/xmodem.o
descr               0x10              ./src/flash.o
rawBuffer           0x100             ./src/xmodem.o

Discarded input sections

 .text          0x00000000        0x0 c:/program files (x86)/gnu tools arm embedded/5.2 2015q4/bin/../lib/gcc/arm-none-eabi/5.2.1/armv6-m/crti.o
 .data          0x00000000        0x0 c:/program files (x86)/gnu tools arm embedded/5.2 2015q4/bin/../lib/gcc/arm-none-eabi/5.2.1/armv6-m/crti.o
 .bss           0x00000000        0x0 c:/program files (x86)/gnu tools arm embedded/5.2 2015q4/bin/../lib/gcc/arm-none-eabi/5.2.1/armv6-m/crti.o
 .data          0x00000000        0x4 c:/program files (x86)/gnu tools arm embedded/5.2 2015q4/bin/../lib/gcc/arm-none-eabi/5.2.1/armv6-m/crtbegin.o
 .data          0x00000000        0x0 c:/program files (x86)/gnu tools arm embedded/5.2 2015q4/bin/../lib/gcc/arm-none-eabi/5.2.1/../../../../arm-none-eabi/lib/armv6-m/crt0.o
 .bss           0x00000000        0x0 c:/program files (x86)/gnu tools arm embedded/5.2 2015q4/bin/../lib/gcc/arm-none-eabi/5.2.1/../../../../arm-none-eabi/lib/armv6-m/crt0.o
 .ARM.extab     0x00000000        0x0 c:/program files (x86)/gnu tools arm embedded/5.2 2015q4/bin/../lib/gcc/arm-none-eabi/5.2.1/../../../../arm-none-eabi/lib/armv6-m/crt0.o
 .text          0x00000000        0x0 ./src/aes.o
 .data          0x00000000        0x0 ./src/aes.o
 .bss           0x00000000        0x0 ./src/aes.o
 .text          0x00000000        0x0 ./src/aes_keys.o
 .data          0x00000000        0x0 ./src/aes_keys.o
 .bss           0x00000000        0x0 ./src/aes_keys.o
 .text          0x00000000        0x0 ./src/boot.o
 .data          0x00000000        0x0 ./src/boot.o
 .bss           0x00000000        0x0 ./src/boot.o
 .text          0x00000000        0x0 ./src/bootloader.o
 .data          0x00000000        0x0 ./src/bootloader.o
 .bss           0x00000000        0x0 ./src/bootloader.o
 .text          0x00000000        0x0 ./src/crc.o
 .data          0x00000000        0x0 ./src/crc.o
 .bss           0x00000000        0x0 ./src/crc.o
 .text          0x00000000        0x0 ./src/debuglock.o
 .data          0x00000000        0x0 ./src/debuglock.o
 .bss           0x00000000        0x0 ./src/debuglock.o
 .text          0x00000000        0x0 ./src/flash.o
 .data          0x00000000        0x0 ./src/flash.o
 .bss           0x00000000        0x0 ./src/flash.o
 .text          0x00000000        0x0 ./src/uart.o
 .data          0x00000000        0x0 ./src/uart.o
 .bss           0x00000000        0x0 ./src/uart.o
 .text          0x00000000        0x0 ./src/verify.o
 .data          0x00000000        0x0 ./src/verify.o
 .bss           0x00000000        0x0 ./src/verify.o
 .text.verifyFirmware
                0x00000000      0x160 ./src/verify.o
 .text          0x00000000        0x0 ./src/xmodem.o
 .data          0x00000000        0x0 ./src/xmodem.o
 .bss           0x00000000        0x0 ./src/xmodem.o
 .text          0x00000000        0x0 ./emlib/em_assert.o
 .data          0x00000000        0x0 ./emlib/em_assert.o
 .bss           0x00000000        0x0 ./emlib/em_assert.o
 .debug_line    0x00000000        0x0 ./emlib/em_assert.o
 .debug_str     0x00000000       0xee ./emlib/em_assert.o
 .comment       0x00000000       0x6f ./emlib/em_assert.o
 .ARM.attributes
                0x00000000       0x32 ./emlib/em_assert.o
 .text          0x00000000        0x0 ./emlib/em_cmu.o
 .data          0x00000000        0x0 ./emlib/em_cmu.o
 .bss           0x00000000        0x0 ./emlib/em_cmu.o
 .text.CMU_AUXHFRCOBandGet
                0x00000000       0x10 ./emlib/em_cmu.o
 .text.CMU_AUXHFRCOBandSet
                0x00000000       0x58 ./emlib/em_cmu.o
 .rodata.CMU_AUXHFRCOBandSet
                0x00000000       0x20 ./emlib/em_cmu.o
 .text.CMU_Calibrate
                0x00000000       0x5c ./emlib/em_cmu.o
 .rodata.CMU_Calibrate
                0x00000000       0x14 ./emlib/em_cmu.o
 .text.CMU_CalibrateConfig
                0x00000000       0x68 ./emlib/em_cmu.o
 .rodata.CMU_CalibrateConfig
                0x00000000       0x14 ./emlib/em_cmu.o
 .text.CMU_CalibrateCountGet
                0x00000000       0x28 ./emlib/em_cmu.o
 .text.CMU_ClockDivGet
                0x00000000       0x74 ./emlib/em_cmu.o
 .rodata.CMU_ClockDivGet
                0x00000000       0x20 ./emlib/em_cmu.o
 .text.CMU_ClockDivSet
                0x00000000      0x164 ./emlib/em_cmu.o
 .rodata.CMU_ClockDivSet
                0x00000000       0x20 ./emlib/em_cmu.o
 .text.CMU_ClockSelectSet
                0x00000000      0x250 ./emlib/em_cmu.o
 .rodata.CMU_ClockSelectSet
                0x00000000       0x7c ./emlib/em_cmu.o
 .text.CMU_FreezeEnable
                0x00000000       0x20 ./emlib/em_cmu.o
 .text.CMU_HFRCOBandGet
                0x00000000       0x10 ./emlib/em_cmu.o
 .text.CMU_HFRCOBandSet
                0x00000000      0x128 ./emlib/em_cmu.o
 .rodata.CMU_HFRCOBandSet
                0x00000000       0x14 ./emlib/em_cmu.o
 .text.CMU_HFRCOStartupDelayGet
                0x00000000       0x10 ./emlib/em_cmu.o
 .text.CMU_HFRCOStartupDelaySet
                0x00000000       0x24 ./emlib/em_cmu.o
 .text.CMU_HFXOInit
                0x00000000       0x40 ./emlib/em_cmu.o
 .text.CMU_LCDClkFDIVGet
                0x00000000        0x4 ./emlib/em_cmu.o
 .text.CMU_LCDClkFDIVSet
                0x00000000        0x4 ./emlib/em_cmu.o
 .text.CMU_LFXOInit
                0x00000000       0x3c ./emlib/em_cmu.o
 .text.CMU_OscillatorEnable
                0x00000000       0x78 ./emlib/em_cmu.o
 .rodata.CMU_OscillatorEnable
                0x00000000       0x18 ./emlib/em_cmu.o
 .text.CMU_OscillatorTuningGet
                0x00000000       0x34 ./emlib/em_cmu.o
 .text.CMU_OscillatorTuningSet
                0x00000000       0x44 ./emlib/em_cmu.o
 .text.CMU_PCNTClockExternalGet
                0x00000000       0x18 ./emlib/em_cmu.o
 .text.CMU_PCNTClockExternalSet
                0x00000000       0x1c ./emlib/em_cmu.o
 .text.CMU_USHFRCOBandGet
                0x00000000       0x10 ./emlib/em_cmu.o
 .text.CMU_USHFRCOBandSet
                0x00000000       0x7c ./emlib/em_cmu.o
 .text          0x00000000        0x0 ./emlib/em_emu.o
 .data          0x00000000        0x0 ./emlib/em_emu.o
 .bss           0x00000000        0x0 ./emlib/em_emu.o
 .text.EMU_EnterEM2
                0x00000000       0x38 ./emlib/em_emu.o
 .text.EMU_EnterEM4
                0x00000000       0x40 ./emlib/em_emu.o
 .text.EMU_MemPwrDown
                0x00000000        0x4 ./emlib/em_emu.o
 .text.EMU_UpdateOscConfig
                0x00000000       0x14 ./emlib/em_emu.o
 .text.EMU_EM23Init
                0x00000000       0x24 ./emlib/em_emu.o
 .text          0x00000000        0x0 ./emlib/em_gpio.o
 .data          0x00000000        0x0 ./emlib/em_gpio.o
 .bss           0x00000000        0x0 ./emlib/em_gpio.o
 .text.GPIO_DbgLocationSet
                0x00000000        0x4 ./emlib/em_gpio.o
 .text.GPIO_DriveModeSet
                0x00000000       0x1c ./emlib/em_gpio.o
 .text.GPIO_PinModeGet
                0x00000000       0x38 ./emlib/em_gpio.o
 .text.GPIO_EM4EnablePinWakeup
                0x00000000       0x3c ./emlib/em_gpio.o
 .text          0x00000000        0x0 ./emlib/em_int.o
 .data          0x00000000        0x0 ./emlib/em_int.o
 .bss           0x00000000        0x0 ./emlib/em_int.o
 .text          0x00000000        0x0 ./emlib/em_msc.o
 .data          0x00000000        0x0 ./emlib/em_msc.o
 .bss           0x00000000        0x0 ./emlib/em_msc.o
 .ram           0x00000000      0x5c4 ./emlib/em_msc.o
 .text.MSC_Init
                0x00000000       0x74 ./emlib/em_msc.o
 .text.MSC_Deinit
                0x00000000       0x14 ./emlib/em_msc.o
 .text.MSC_ExecConfigSet
                0x00000000       0x28 ./emlib/em_msc.o
 .debug_info    0x00000000      0xce2 ./emlib/em_msc.o
 .debug_abbrev  0x00000000      0x320 ./emlib/em_msc.o
 .debug_loc     0x00000000     0x1346 ./emlib/em_msc.o
 .debug_aranges
                0x00000000       0x80 ./emlib/em_msc.o
 .debug_ranges  0x00000000      0x298 ./emlib/em_msc.o
 .debug_line    0x00000000      0x5b2 ./emlib/em_msc.o
 .debug_str     0x00000000      0x6a3 ./emlib/em_msc.o
 .comment       0x00000000       0x6f ./emlib/em_msc.o
 .debug_frame   0x00000000      0x160 ./emlib/em_msc.o
 .ARM.attributes
                0x00000000       0x32 ./emlib/em_msc.o
 .text          0x00000000        0x0 ./emlib/em_system.o
 .data          0x00000000        0x0 ./emlib/em_system.o
 .bss           0x00000000        0x0 ./emlib/em_system.o
 .text.SYSTEM_ChipRevisionGet
                0x00000000       0x34 ./emlib/em_system.o
 .text.SYSTEM_GetCalibrationValue
                0x00000000       0x28 ./emlib/em_system.o
 .debug_info    0x00000000      0x257 ./emlib/em_system.o
 .debug_abbrev  0x00000000       0xdc ./emlib/em_system.o
 .debug_loc     0x00000000       0xcc ./emlib/em_system.o
 .debug_aranges
                0x00000000       0x28 ./emlib/em_system.o
 .debug_ranges  0x00000000       0x18 ./emlib/em_system.o
 .debug_line    0x00000000      0x21c ./emlib/em_system.o
 .debug_str     0x00000000      0x292 ./emlib/em_system.o
 .comment       0x00000000       0x6f ./emlib/em_system.o
 .debug_frame   0x00000000       0x38 ./emlib/em_system.o
 .ARM.attributes
                0x00000000       0x32 ./emlib/em_system.o
 .text          0x00000000        0x0 ./emlib/em_usart.o
 .data          0x00000000        0x0 ./emlib/em_usart.o
 .bss           0x00000000        0x0 ./emlib/em_usart.o
 .text.USART_BaudrateAsyncSet
                0x00000000       0x68 ./emlib/em_usart.o
 .text.USART_BaudrateCalc
                0x00000000       0x8c ./emlib/em_usart.o
 .text.USART_BaudrateGet
                0x00000000       0xc0 ./emlib/em_usart.o
 .text.USART_BaudrateSyncSet
                0x00000000       0x40 ./emlib/em_usart.o
 .text.USART_Enable
                0x00000000       0x10 ./emlib/em_usart.o
 .text.USART_InitSync
                0x00000000       0xd0 ./emlib/em_usart.o
 .text.USARTn_InitIrDA
                0x00000000      0x118 ./emlib/em_usart.o
 .text.USART_InitI2s
                0x00000000      0x110 ./emlib/em_usart.o
 .text.USART_InitPrsTrigger
                0x00000000       0x2c ./emlib/em_usart.o
 .text.USART_Reset
                0x00000000       0x48 ./emlib/em_usart.o
 .text.USART_Rx
                0x00000000       0x10 ./emlib/em_usart.o
 .text.USART_RxDouble
                0x00000000       0x10 ./emlib/em_usart.o
 .text.USART_RxDoubleExt
                0x00000000       0x10 ./emlib/em_usart.o
 .text.USART_RxExt
                0x00000000       0x10 ./emlib/em_usart.o
 .text.USART_SpiTransfer
                0x00000000       0x18 ./emlib/em_usart.o
 .text.USART_Tx
                0x00000000        0xc ./emlib/em_usart.o
 .text.USART_TxDouble
                0x00000000        0xc ./emlib/em_usart.o
 .text.USART_TxDoubleExt
                0x00000000        0xc ./emlib/em_usart.o
 .text.USART_TxExt
                0x00000000        0xc ./emlib/em_usart.o
 .data          0x00000000        0x0 ./CMSIS/efm32hg/startup_efm32hg.o
 .bss           0x00000000        0x0 ./CMSIS/efm32hg/startup_efm32hg.o
 .text          0x00000000        0x0 ./CMSIS/efm32hg/system_efm32hg.o
 .data          0x00000000        0x0 ./CMSIS/efm32hg/system_efm32hg.o
 .bss           0x00000000        0x0 ./CMSIS/efm32hg/system_efm32hg.o
 .text.SystemMaxCoreClockGet
                0x00000000        0x8 ./CMSIS/efm32hg/system_efm32hg.o
 .text.SystemHFXOClockGet
                0x00000000        0xc ./CMSIS/efm32hg/system_efm32hg.o
 .text.SystemHFXOClockSet
                0x00000000       0xd8 ./CMSIS/efm32hg/system_efm32hg.o
 .text.SystemLFXOClockSet
                0x00000000       0xd8 ./CMSIS/efm32hg/system_efm32hg.o
 .data          0x00000000        0x0 c:/program files (x86)/gnu tools arm embedded/5.2 2015q4/bin/../lib/gcc/arm-none-eabi/5.2.1/armv6-m\libgcc.a(_udivsi3.o)
 .bss           0x00000000        0x0 c:/program files (x86)/gnu tools arm embedded/5.2 2015q4/bin/../lib/gcc/arm-none-eabi/5.2.1/armv6-m\libgcc.a(_udivsi3.o)
 .data          0x00000000        0x0 c:/program files (x86)/gnu tools arm embedded/5.2 2015q4/bin/../lib/gcc/arm-none-eabi/5.2.1/armv6-m\libgcc.a(_dvmd_tls.o)
 .bss           0x00000000        0x0 c:/program files (x86)/gnu tools arm embedded/5.2 2015q4/bin/../lib/gcc/arm-none-eabi/5.2.1/armv6-m\libgcc.a(_dvmd_tls.o)
 .text          0x00000000       0x3c c:/program files (x86)/gnu tools arm embedded/5.2 2015q4/bin/../lib/gcc/arm-none-eabi/5.2.1/armv6-m\libgcc.a(_clzsi2.o)
 .data          0x00000000        0x0 c:/program files (x86)/gnu tools arm embedded/5.2 2015q4/bin/../lib/gcc/arm-none-eabi/5.2.1/armv6-m\libgcc.a(_clzsi2.o)
 .bss           0x00000000        0x0 c:/program files (x86)/gnu tools arm embedded/5.2 2015q4/bin/../lib/gcc/arm-none-eabi/5.2.1/armv6-m\libgcc.a(_clzsi2.o)
 .ARM.attributes
                0x00000000       0x1e c:/program files (x86)/gnu tools arm embedded/5.2 2015q4/bin/../lib/gcc/arm-none-eabi/5.2.1/armv6-m\libgcc.a(_clzsi2.o)
 .text          0x00000000       0x40 c:/program files (x86)/gnu tools arm embedded/5.2 2015q4/bin/../lib/gcc/arm-none-eabi/5.2.1/armv6-m\libgcc.a(_aeabi_uldivmod.o)
 .data          0x00000000        0x0 c:/program files (x86)/gnu tools arm embedded/5.2 2015q4/bin/../lib/gcc/arm-none-eabi/5.2.1/armv6-m\libgcc.a(_aeabi_uldivmod.o)
 .bss           0x00000000        0x0 c:/program files (x86)/gnu tools arm embedded/5.2 2015q4/bin/../lib/gcc/arm-none-eabi/5.2.1/armv6-m\libgcc.a(_aeabi_uldivmod.o)
 .ARM.attributes
                0x00000000       0x1e c:/program files (x86)/gnu tools arm embedded/5.2 2015q4/bin/../lib/gcc/arm-none-eabi/5.2.1/armv6-m\libgcc.a(_aeabi_uldivmod.o)
 .text          0x00000000       0x58 c:/program files (x86)/gnu tools arm embedded/5.2 2015q4/bin/../lib/gcc/arm-none-eabi/5.2.1/armv6-m\libgcc.a(_muldi3.o)
 .data          0x00000000        0x0 c:/program files (x86)/gnu tools arm embedded/5.2 2015q4/bin/../lib/gcc/arm-none-eabi/5.2.1/armv6-m\libgcc.a(_muldi3.o)
 .bss           0x00000000        0x0 c:/program files (x86)/gnu tools arm embedded/5.2 2015q4/bin/../lib/gcc/arm-none-eabi/5.2.1/armv6-m\libgcc.a(_muldi3.o)
 .debug_frame   0x00000000       0x34 c:/program files (x86)/gnu tools arm embedded/5.2 2015q4/bin/../lib/gcc/arm-none-eabi/5.2.1/armv6-m\libgcc.a(_muldi3.o)
 .ARM.attributes
                0x00000000       0x2c c:/program files (x86)/gnu tools arm embedded/5.2 2015q4/bin/../lib/gcc/arm-none-eabi/5.2.1/armv6-m\libgcc.a(_muldi3.o)
 .text          0x00000000      0x180 c:/program files (x86)/gnu tools arm embedded/5.2 2015q4/bin/../lib/gcc/arm-none-eabi/5.2.1/armv6-m\libgcc.a(_udivmoddi4.o)
 .data          0x00000000        0x0 c:/program files (x86)/gnu tools arm embedded/5.2 2015q4/bin/../lib/gcc/arm-none-eabi/5.2.1/armv6-m\libgcc.a(_udivmoddi4.o)
 .bss           0x00000000        0x0 c:/program files (x86)/gnu tools arm embedded/5.2 2015q4/bin/../lib/gcc/arm-none-eabi/5.2.1/armv6-m\libgcc.a(_udivmoddi4.o)
 .ARM.extab     0x00000000        0x0 c:/program files (x86)/gnu tools arm embedded/5.2 2015q4/bin/../lib/gcc/arm-none-eabi/5.2.1/armv6-m\libgcc.a(_udivmoddi4.o)
 .ARM.exidx     0x00000000        0x8 c:/program files (x86)/gnu tools arm embedded/5.2 2015q4/bin/../lib/gcc/arm-none-eabi/5.2.1/armv6-m\libgcc.a(_udivmoddi4.o)
 .debug_frame   0x00000000       0x3c c:/program files (x86)/gnu tools arm embedded/5.2 2015q4/bin/../lib/gcc/arm-none-eabi/5.2.1/armv6-m\libgcc.a(_udivmoddi4.o)
 .ARM.attributes
                0x00000000       0x2c c:/program files (x86)/gnu tools arm embedded/5.2 2015q4/bin/../lib/gcc/arm-none-eabi/5.2.1/armv6-m\libgcc.a(_udivmoddi4.o)
 .text          0x00000000       0x18 c:/program files (x86)/gnu tools arm embedded/5.2 2015q4/bin/../lib/gcc/arm-none-eabi/5.2.1/armv6-m\libgcc.a(_clzdi2.o)
 .data          0x00000000        0x0 c:/program files (x86)/gnu tools arm embedded/5.2 2015q4/bin/../lib/gcc/arm-none-eabi/5.2.1/armv6-m\libgcc.a(_clzdi2.o)
 .bss           0x00000000        0x0 c:/program files (x86)/gnu tools arm embedded/5.2 2015q4/bin/../lib/gcc/arm-none-eabi/5.2.1/armv6-m\libgcc.a(_clzdi2.o)
 .ARM.attributes
                0x00000000       0x1e c:/program files (x86)/gnu tools arm embedded/5.2 2015q4/bin/../lib/gcc/arm-none-eabi/5.2.1/armv6-m\libgcc.a(_clzdi2.o)
 .text          0x00000000        0x0 c:/program files (x86)/gnu tools arm embedded/5.2 2015q4/bin/../lib/gcc/arm-none-eabi/5.2.1/../../../../arm-none-eabi/lib/armv6-m\libc_nano.a(lib_a-exit.o)
 .data          0x00000000        0x0 c:/program files (x86)/gnu tools arm embedded/5.2 2015q4/bin/../lib/gcc/arm-none-eabi/5.2.1/../../../../arm-none-eabi/lib/armv6-m\libc_nano.a(lib_a-exit.o)
 .bss           0x00000000        0x0 c:/program files (x86)/gnu tools arm embedded/5.2 2015q4/bin/../lib/gcc/arm-none-eabi/5.2.1/../../../../arm-none-eabi/lib/armv6-m\libc_nano.a(lib_a-exit.o)
 .text          0x00000000        0x0 c:/program files (x86)/gnu tools arm embedded/5.2 2015q4/bin/../lib/gcc/arm-none-eabi/5.2.1/../../../../arm-none-eabi/lib/armv6-m\libc_nano.a(lib_a-impure.o)
 .data          0x00000000        0x0 c:/program files (x86)/gnu tools arm embedded/5.2 2015q4/bin/../lib/gcc/arm-none-eabi/5.2.1/../../../../arm-none-eabi/lib/armv6-m\libc_nano.a(lib_a-impure.o)
 .bss           0x00000000        0x0 c:/program files (x86)/gnu tools arm embedded/5.2 2015q4/bin/../lib/gcc/arm-none-eabi/5.2.1/../../../../arm-none-eabi/lib/armv6-m\libc_nano.a(lib_a-impure.o)
 .data._impure_ptr
                0x00000000        0x4 c:/program files (x86)/gnu tools arm embedded/5.2 2015q4/bin/../lib/gcc/arm-none-eabi/5.2.1/../../../../arm-none-eabi/lib/armv6-m\libc_nano.a(lib_a-impure.o)
 .text          0x00000000        0x0 c:/program files (x86)/gnu tools arm embedded/5.2 2015q4/bin/../lib/gcc/arm-none-eabi/5.2.1/../../../../arm-none-eabi/lib/armv6-m\libc_nano.a(lib_a-init.o)
 .data          0x00000000        0x0 c:/program files (x86)/gnu tools arm embedded/5.2 2015q4/bin/../lib/gcc/arm-none-eabi/5.2.1/../../../../arm-none-eabi/lib/armv6-m\libc_nano.a(lib_a-init.o)
 .bss           0x00000000        0x0 c:/program files (x86)/gnu tools arm embedded/5.2 2015q4/bin/../lib/gcc/arm-none-eabi/5.2.1/../../../../arm-none-eabi/lib/armv6-m\libc_nano.a(lib_a-init.o)
 .text          0x00000000        0x0 c:/program files (x86)/gnu tools arm embedded/5.2 2015q4/bin/../lib/gcc/arm-none-eabi/5.2.1/../../../../arm-none-eabi/lib/armv6-m\libc_nano.a(lib_a-memcpy-stub.o)
 .data          0x00000000        0x0 c:/program files (x86)/gnu tools arm embedded/5.2 2015q4/bin/../lib/gcc/arm-none-eabi/5.2.1/../../../../arm-none-eabi/lib/armv6-m\libc_nano.a(lib_a-memcpy-stub.o)
 .bss           0x00000000        0x0 c:/program files (x86)/gnu tools arm embedded/5.2 2015q4/bin/../lib/gcc/arm-none-eabi/5.2.1/../../../../arm-none-eabi/lib/armv6-m\libc_nano.a(lib_a-memcpy-stub.o)
 .text          0x00000000        0x0 c:/program files (x86)/gnu tools arm embedded/5.2 2015q4/bin/../lib/gcc/arm-none-eabi/5.2.1/../../../../arm-none-eabi/lib/armv6-m\libc_nano.a(lib_a-memset.o)
 .data          0x00000000        0x0 c:/program files (x86)/gnu tools arm embedded/5.2 2015q4/bin/../lib/gcc/arm-none-eabi/5.2.1/../../../../arm-none-eabi/lib/armv6-m\libc_nano.a(lib_a-memset.o)
 .bss           0x00000000        0x0 c:/program files (x86)/gnu tools arm embedded/5.2 2015q4/bin/../lib/gcc/arm-none-eabi/5.2.1/../../../../arm-none-eabi/lib/armv6-m\libc_nano.a(lib_a-memset.o)
 .text          0x00000000        0x0 c:/program files (x86)/gnu tools arm embedded/5.2 2015q4/bin/../lib/gcc/arm-none-eabi/5.2.1/../../../../arm-none-eabi/lib/armv6-m\libnosys.a(_exit.o)
 .data          0x00000000        0x0 c:/program files (x86)/gnu tools arm embedded/5.2 2015q4/bin/../lib/gcc/arm-none-eabi/5.2.1/../../../../arm-none-eabi/lib/armv6-m\libnosys.a(_exit.o)
 .bss           0x00000000        0x0 c:/program files (x86)/gnu tools arm embedded/5.2 2015q4/bin/../lib/gcc/arm-none-eabi/5.2.1/../../../../arm-none-eabi/lib/armv6-m\libnosys.a(_exit.o)
 .text          0x00000000        0x0 c:/program files (x86)/gnu tools arm embedded/5.2 2015q4/bin/../lib/gcc/arm-none-eabi/5.2.1/armv6-m/crtend.o
 .data          0x00000000        0x0 c:/program files (x86)/gnu tools arm embedded/5.2 2015q4/bin/../lib/gcc/arm-none-eabi/5.2.1/armv6-m/crtend.o
 .bss           0x00000000        0x0 c:/program files (x86)/gnu tools arm embedded/5.2 2015q4/bin/../lib/gcc/arm-none-eabi/5.2.1/armv6-m/crtend.o
 .text          0x00000000        0x0 c:/program files (x86)/gnu tools arm embedded/5.2 2015q4/bin/../lib/gcc/arm-none-eabi/5.2.1/armv6-m/crtn.o
 .data          0x00000000        0x0 c:/program files (x86)/gnu tools arm embedded/5.2 2015q4/bin/../lib/gcc/arm-none-eabi/5.2.1/armv6-m/crtn.o
 .bss           0x00000000        0x0 c:/program files (x86)/gnu tools arm embedded/5.2 2015q4/bin/../lib/gcc/arm-none-eabi/5.2.1/armv6-m/crtn.o

Memory Configuration

Name             Origin             Length             Attributes
FLASH            0x00000000         0x00004000         xr
RAM              0x20000000         0x00002000         xrw
*default*        0x00000000         0xffffffff

Linker script and memory map

LOAD c:/program files (x86)/gnu tools arm embedded/5.2 2015q4/bin/../lib/gcc/arm-none-eabi/5.2.1/armv6-m/crti.o
LOAD c:/program files (x86)/gnu tools arm embedded/5.2 2015q4/bin/../lib/gcc/arm-none-eabi/5.2.1/armv6-m/crtbegin.o
LOAD c:/program files (x86)/gnu tools arm embedded/5.2 2015q4/bin/../lib/gcc/arm-none-eabi/5.2.1/../../../../arm-none-eabi/lib/armv6-m/crt0.o
LOAD ./src/aes.o
LOAD ./src/aes_keys.o
LOAD ./src/boot.o
LOAD ./src/bootloader.o
LOAD ./src/crc.o
LOAD ./src/debuglock.o
LOAD ./src/flash.o
LOAD ./src/uart.o
LOAD ./src/verify.o
LOAD ./src/xmodem.o
LOAD ./emlib/em_assert.o
LOAD ./emlib/em_cmu.o
LOAD ./emlib/em_emu.o
LOAD ./emlib/em_gpio.o
LOAD ./emlib/em_int.o
LOAD ./emlib/em_msc.o
LOAD ./emlib/em_system.o
LOAD ./emlib/em_usart.o
LOAD ./CMSIS/efm32hg/startup_efm32hg.o
LOAD ./CMSIS/efm32hg/system_efm32hg.o
START GROUP
LOAD c:/program files (x86)/gnu tools arm embedded/5.2 2015q4/bin/../lib/gcc/arm-none-eabi/5.2.1/armv6-m\libgcc.a
LOAD c:/program files (x86)/gnu tools arm embedded/5.2 2015q4/bin/../lib/gcc/arm-none-eabi/5.2.1/../../../../arm-none-eabi/lib/armv6-m\libc_nano.a
LOAD c:/program files (x86)/gnu tools arm embedded/5.2 2015q4/bin/../lib/gcc/arm-none-eabi/5.2.1/../../../../arm-none-eabi/lib/armv6-m\libnosys.a
END GROUP
START GROUP
LOAD c:/program files (x86)/gnu tools arm embedded/5.2 2015q4/bin/../lib/gcc/arm-none-eabi/5.2.1/armv6-m\libgcc.a
LOAD c:/program files (x86)/gnu tools arm embedded/5.2 2015q4/bin/../lib/gcc/arm-none-eabi/5.2.1/../../../../arm-none-eabi/lib/armv6-m\libg_nano.a
LOAD c:/program files (x86)/gnu tools arm embedded/5.2 2015q4/bin/../lib/gcc/arm-none-eabi/5.2.1/../../../../arm-none-eabi/lib/armv6-m\libc_nano.a
END GROUP
START GROUP
LOAD c:/program files (x86)/gnu tools arm embedded/5.2 2015q4/bin/../lib/gcc/arm-none-eabi/5.2.1/armv6-m\libgcc.a
LOAD c:/program files (x86)/gnu tools arm embedded/5.2 2015q4/bin/../lib/gcc/arm-none-eabi/5.2.1/../../../../arm-none-eabi/lib/armv6-m\libc_nano.a
END GROUP
LOAD c:/program files (x86)/gnu tools arm embedded/5.2 2015q4/bin/../lib/gcc/arm-none-eabi/5.2.1/armv6-m/crtend.o
LOAD c:/program files (x86)/gnu tools arm embedded/5.2 2015q4/bin/../lib/gcc/arm-none-eabi/5.2.1/armv6-m/crtn.o

.text           0x00000000     0x1688
 *(.vectors)
 .vectors       0x00000000       0x94 ./CMSIS/efm32hg/startup_efm32hg.o
                0x00000000                __Vectors
                0x00000094                __Vectors_End = .
                0x00000094                __Vectors_Size = (__Vectors_End - __Vectors)
                0x00000094                __end__ = .
 *(.text*)
 .text          0x00000094       0xb4 c:/program files (x86)/gnu tools arm embedded/5.2 2015q4/bin/../lib/gcc/arm-none-eabi/5.2.1/armv6-m/crtbegin.o
 .text          0x00000148       0x78 c:/program files (x86)/gnu tools arm embedded/5.2 2015q4/bin/../lib/gcc/arm-none-eabi/5.2.1/../../../../arm-none-eabi/lib/armv6-m/crt0.o
                0x00000148                _start
                0x00000148                _mainCRTStartup
 .text.BOOT_jump
                0x000001c0       0x1c ./src/boot.o
                0x000001c0                BOOT_jump
 .text.BOOT_boot
                0x000001dc       0x30 ./src/boot.o
                0x000001dc                BOOT_boot
 .text.sendWelcomeMessage
                0x0000020c       0x78 ./src/bootloader.o
                0x0000020c                sendWelcomeMessage
 .text.enterDownloadMode
                0x00000284       0x98 ./src/bootloader.o
                0x00000284                enterDownloadMode
 .text.enableDebugLock
                0x0000031c       0x24 ./src/bootloader.o
                0x0000031c                enableDebugLock
 .text.commandLoop
                0x00000340       0x9c ./src/bootloader.o
                0x00000340                commandLoop
 .text.GPIO_EVEN_IRQHandler
                0x000003dc       0x14 ./src/bootloader.o
                0x000003dc                GPIO_EVEN_IRQHandler
 .text.GPIO_ODD_IRQHandler
                0x000003f0       0x14 ./src/bootloader.o
                0x000003f0                GPIO_ODD_IRQHandler
 .text.enterLowPowerWait
                0x00000404       0x58 ./src/bootloader.o
                0x00000404                enterLowPowerWait
 .text.enterBootloaderMode
                0x0000045c       0x3c ./src/bootloader.o
                0x0000045c                enterBootloaderMode
 .text.startup.main
                0x00000498       0x98 ./src/bootloader.o
                0x00000498                main
 .text.BLUART_init
                0x00000530       0x60 ./src/uart.o
                0x00000530                BLUART_init
 .text.verifyActiveFirmware
                0x00000590      0x148 ./src/verify.o
                0x00000590                verifyActiveFirmware
 .text.verifyTempStorage
                0x000006d8      0x148 ./src/verify.o
                0x000006d8                verifyTempStorage
 .text.isFirmwareValid
                0x00000820       0x18 ./src/verify.o
                0x00000820                isFirmwareValid
 .text.isTempStorageValid
                0x00000838       0x18 ./src/verify.o
                0x00000838                isTempStorageValid
 .text.markFirmwareAsVerified
                0x00000850       0x14 ./src/verify.o
                0x00000850                markFirmwareAsVerified
 .text.markTempAsVerified
                0x00000864       0x14 ./src/verify.o
                0x00000864                markTempAsVerified
 .text.markFirmwareAsDeleted
                0x00000878       0x10 ./src/verify.o
                0x00000878                markFirmwareAsDeleted
 .text.CMU_ClockEnable
                0x00000888       0x88 ./emlib/em_cmu.o
                0x00000888                CMU_ClockEnable
 .text.CMU_ClockSelectGet
                0x00000910       0xe8 ./emlib/em_cmu.o
                0x00000910                CMU_ClockSelectGet
 .text.CMU_ClockFreqGet
                0x000009f8      0x254 ./emlib/em_cmu.o
                0x000009f8                CMU_ClockFreqGet
 .text.emuRestore
                0x00000c4c       0xd4 ./emlib/em_emu.o
 .text.EMU_EnterEM3
                0x00000d20       0x54 ./emlib/em_emu.o
                0x00000d20                EMU_EnterEM3
 .text.GPIO_ExtIntConfig
                0x00000d74       0xa0 ./emlib/em_gpio.o
                0x00000d74                GPIO_ExtIntConfig
 .text.GPIO_PinModeSet
                0x00000e14       0xa4 ./emlib/em_gpio.o
                0x00000e14                GPIO_PinModeSet
 .text.USART_InitAsync
                0x00000eb8       0xdc ./emlib/em_usart.o
                0x00000eb8                USART_InitAsync
 .text          0x00000f94       0x30 ./CMSIS/efm32hg/startup_efm32hg.o
                0x00000f94                Reset_Handler
                0x00000fc0                USART0_TX_IRQHandler
                0x00000fc0                I2C0_IRQHandler
                0x00000fc0                HardFault_Handler
                0x00000fc0                SysTick_Handler
                0x00000fc0                USART1_RX_IRQHandler
                0x00000fc0                PendSV_Handler
                0x00000fc0                NMI_Handler
                0x00000fc0                USART1_TX_IRQHandler
                0x00000fc0                MSC_IRQHandler
                0x00000fc0                ADC0_IRQHandler
                0x00000fc0                LEUART0_IRQHandler
                0x00000fc0                RTC_IRQHandler
                0x00000fc0                TIMER0_IRQHandler
                0x00000fc0                TIMER2_IRQHandler
                0x00000fc0                TIMER1_IRQHandler
                0x00000fc0                Default_Handler
                0x00000fc0                PCNT0_IRQHandler
                0x00000fc0                USB_IRQHandler
                0x00000fc0                ACMP0_IRQHandler
                0x00000fc0                USART0_RX_IRQHandler
                0x00000fc0                SVC_Handler
                0x00000fc0                CMU_IRQHandler
                0x00000fc0                AES_IRQHandler
                0x00000fc0                VCMP_IRQHandler
                0x00000fc0                DMA_IRQHandler
 .text.SystemCoreClockGet
                0x00000fc4       0xd0 ./CMSIS/efm32hg/system_efm32hg.o
                0x00000fc4                SystemCoreClockGet
 .text.SystemHFClockGet
                0x00001094       0xc0 ./CMSIS/efm32hg/system_efm32hg.o
                0x00001094                SystemHFClockGet
 .text.SystemInit
                0x00001154        0x4 ./CMSIS/efm32hg/system_efm32hg.o
                0x00001154                SystemInit
 .text.SystemLFRCOClockGet
                0x00001158        0x8 ./CMSIS/efm32hg/system_efm32hg.o
                0x00001158                SystemLFRCOClockGet
 .text.SystemULFRCOClockGet
                0x00001160        0x8 ./CMSIS/efm32hg/system_efm32hg.o
                0x00001160                SystemULFRCOClockGet
 .text.SystemLFXOClockGet
                0x00001168        0xc ./CMSIS/efm32hg/system_efm32hg.o
                0x00001168                SystemLFXOClockGet
 .text          0x00001174      0x114 c:/program files (x86)/gnu tools arm embedded/5.2 2015q4/bin/../lib/gcc/arm-none-eabi/5.2.1/armv6-m\libgcc.a(_udivsi3.o)
                0x00001174                __aeabi_uidiv
                0x00001174                __udivsi3
                0x00001280                __aeabi_uidivmod
 .text          0x00001288        0x4 c:/program files (x86)/gnu tools arm embedded/5.2 2015q4/bin/../lib/gcc/arm-none-eabi/5.2.1/armv6-m\libgcc.a(_dvmd_tls.o)
                0x00001288                __aeabi_idiv0
                0x00001288                __aeabi_ldiv0
 .text.exit     0x0000128c       0x2c c:/program files (x86)/gnu tools arm embedded/5.2 2015q4/bin/../lib/gcc/arm-none-eabi/5.2.1/../../../../arm-none-eabi/lib/armv6-m\libc_nano.a(lib_a-exit.o)
                0x0000128c                exit
 .text.__libc_init_array
                0x000012b8       0x4c c:/program files (x86)/gnu tools arm embedded/5.2 2015q4/bin/../lib/gcc/arm-none-eabi/5.2.1/../../../../arm-none-eabi/lib/armv6-m\libc_nano.a(lib_a-init.o)
                0x000012b8                __libc_init_array
 .text.memcpy   0x00001304       0x12 c:/program files (x86)/gnu tools arm embedded/5.2 2015q4/bin/../lib/gcc/arm-none-eabi/5.2.1/../../../../arm-none-eabi/lib/armv6-m\libc_nano.a(lib_a-memcpy-stub.o)
                0x00001304                memcpy
 .text.memset   0x00001316       0x10 c:/program files (x86)/gnu tools arm embedded/5.2 2015q4/bin/../lib/gcc/arm-none-eabi/5.2.1/../../../../arm-none-eabi/lib/armv6-m\libc_nano.a(lib_a-memset.o)
                0x00001316                memset
 *fill*         0x00001326        0x2 
 .text._exit    0x00001328        0x4 c:/program files (x86)/gnu tools arm embedded/5.2 2015q4/bin/../lib/gcc/arm-none-eabi/5.2.1/../../../../arm-none-eabi/lib/armv6-m\libnosys.a(_exit.o)
                0x00001328                _exit
 *(.init)
 .init          0x0000132c        0x4 c:/program files (x86)/gnu tools arm embedded/5.2 2015q4/bin/../lib/gcc/arm-none-eabi/5.2.1/armv6-m/crti.o
                0x0000132c                _init
 .init          0x00001330        0x8 c:/program files (x86)/gnu tools arm embedded/5.2 2015q4/bin/../lib/gcc/arm-none-eabi/5.2.1/armv6-m/crtn.o
 *(.fini)
 .fini          0x00001338        0x4 c:/program files (x86)/gnu tools arm embedded/5.2 2015q4/bin/../lib/gcc/arm-none-eabi/5.2.1/armv6-m/crti.o
                0x00001338                _fini
 .fini          0x0000133c        0x8 c:/program files (x86)/gnu tools arm embedded/5.2 2015q4/bin/../lib/gcc/arm-none-eabi/5.2.1/armv6-m/crtn.o
 *fill*         0x00001344        0x4 
 .fini.__stub   0x00001348       0x80 linker stubs
 *crtbegin.o(.ctors)
 *crtbegin?.o(.ctors)
 *(EXCLUDE_FILE(*crtend.o *crtend?.o) .ctors)
 *(SORT(.ctors.*))
 *(.ctors)
 *crtbegin.o(.dtors)
 *crtbegin?.o(.dtors)
 *(EXCLUDE_FILE(*crtend.o *crtend?.o) .dtors)
 *(SORT(.dtors.*))
 *(.dtors)
 *(.rodata*)
 .rodata.commandLoop
                0x000013c8       0x3c ./src/bootloader.o
 .rodata.str1.4
                0x00001404      0x214 ./src/bootloader.o
 .rodata        0x00001618       0x18 ./src/uart.o
 .rodata.CMU_ClockEnable
                0x00001630       0x2c ./emlib/em_cmu.o
 .rodata.CMU_ClockSelectGet
                0x0000165c       0x20 ./emlib/em_cmu.o
 .rodata.str1.1
                0x0000167c        0x2 c:/program files (x86)/gnu tools arm embedded/5.2 2015q4/bin/../lib/gcc/arm-none-eabi/5.2.1/../../../../arm-none-eabi/lib/armv6-m\libc_nano.a(lib_a-impure.o)
 *fill*         0x0000167e        0x2 
 .rodata._global_impure_ptr
                0x00001680        0x4 c:/program files (x86)/gnu tools arm embedded/5.2 2015q4/bin/../lib/gcc/arm-none-eabi/5.2.1/../../../../arm-none-eabi/lib/armv6-m\libc_nano.a(lib_a-impure.o)
                0x00001680                _global_impure_ptr
 *(.eh_frame*)
 .eh_frame      0x00001684        0x0 c:/program files (x86)/gnu tools arm embedded/5.2 2015q4/bin/../lib/gcc/arm-none-eabi/5.2.1/armv6-m/crtbegin.o
 .eh_frame      0x00001684        0x4 c:/program files (x86)/gnu tools arm embedded/5.2 2015q4/bin/../lib/gcc/arm-none-eabi/5.2.1/armv6-m/crtend.o

.glue_7         0x00001688        0x0
 .glue_7        0x00001688        0x0 linker stubs

.glue_7t        0x00001688        0x0
 .glue_7t       0x00001688        0x0 linker stubs

.vfp11_veneer   0x00001688        0x0
 .vfp11_veneer  0x00001688        0x0 linker stubs

.v4_bx          0x00001688        0x0
 .v4_bx         0x00001688        0x0 linker stubs

.iplt           0x00001688        0x0
 .iplt          0x00001688        0x0 c:/program files (x86)/gnu tools arm embedded/5.2 2015q4/bin/../lib/gcc/arm-none-eabi/5.2.1/armv6-m/crtbegin.o

.ARM.extab
 *(.ARM.extab* .gnu.linkonce.armextab.*)
                0x00001688                __exidx_start = .

.ARM.exidx      0x00001688        0x8
 *(.ARM.exidx* .gnu.linkonce.armexidx.*)
 .ARM.exidx     0x00001688        0x8 c:/program files (x86)/gnu tools arm embedded/5.2 2015q4/bin/../lib/gcc/arm-none-eabi/5.2.1/../../../../arm-none-eabi/lib/armv6-m/crt0.o
                0x00001690                __exidx_end = .
                0x00001690                __etext = .

.rel.dyn        0x00001690        0x0
 .rel.iplt      0x00001690        0x0 c:/program files (x86)/gnu tools arm embedded/5.2 2015q4/bin/../lib/gcc/arm-none-eabi/5.2.1/armv6-m/crtbegin.o

.data           0x20000000      0x9c4 load address 0x00001690
                0x20000000                __data_start__ = .
 *(vtable)
 *(.data*)
 .data.initVector
                0x20000000       0x10 ./src/aes_keys.o
                0x20000000                initVector
 .data.encryptionKey
                0x20000010       0x10 ./src/aes_keys.o
                0x20000010                encryptionKey
 .data.hashInitVector
                0x20000020       0x10 ./src/aes_keys.o
                0x20000020                hashInitVector
 .data.hashKey  0x20000030       0x10 ./src/aes_keys.o
                0x20000030                hashKey
 .data._DEBUGLOCK_swData
                0x20000040       0x15 ./src/debuglock.o
                0x20000040                _DEBUGLOCK_swData
 *fill*         0x20000055        0x3 
 .data.SystemLFXOClock
                0x20000058        0x4 ./CMSIS/efm32hg/system_efm32hg.o
 .data.SystemHFXOClock
                0x2000005c        0x4 ./CMSIS/efm32hg/system_efm32hg.o
 .data.impure_data
                0x20000060       0x60 c:/program files (x86)/gnu tools arm embedded/5.2 2015q4/bin/../lib/gcc/arm-none-eabi/5.2.1/../../../../arm-none-eabi/lib/armv6-m\libc_nano.a(lib_a-impure.o)
                0x200000c0                . = ALIGN (0x4)
 *(.ram)
 .ram           0x200000c0      0x2a8 ./src/aes.o
                0x200000c0                decryptCBC
                0x20000134                encryptCBC128
                0x200001ac                startDecryptCBC
                0x20000270                decryptBlockCBC
                0x20000358                endDecryptCBC
 .ram           0x20000368       0x34 ./src/crc.o
                0x20000368                CRC_calc
 .ram           0x2000039c      0x1e8 ./src/debuglock.o
                0x2000039c                DEBUGLOCK_startDebugInterface
                0x20000528                DEBUGLOCK_lock
                0x20000544                _DEBUGLOCK_driveBit
 .ram           0x20000584      0x218 ./src/flash.o
                0x20000584                FLASH_init
                0x200005bc                FLASH_write
                0x2000061c                FLASH_erasePage
                0x20000654                FLASH_writeWord
                0x2000067c                copyFirmwareFromTempStorage
 .ram           0x2000079c       0x5c ./src/uart.o
                0x2000079c                BLUART_receive
                0x200007b4                BLUART_send
                0x200007c8                BLUART_sendString
 .ram           0x200007f8      0x1b0 ./src/xmodem.o
                0x200007f8                XMODEM_download
                0x2000096c                XMODEM_verifyPacketChecksum
 .ram.__stub    0x200009a8       0x10 linker stubs
                0x200009b8                . = ALIGN (0x4)
                0x200009b8                PROVIDE (__preinit_array_start, .)
 *(.preinit_array)
                0x200009b8                PROVIDE (__preinit_array_end, .)
                0x200009b8                . = ALIGN (0x4)
                0x200009b8                PROVIDE (__init_array_start, .)
 *(SORT(.init_array.*))
 *(.init_array)
 .init_array    0x200009b8        0x4 c:/program files (x86)/gnu tools arm embedded/5.2 2015q4/bin/../lib/gcc/arm-none-eabi/5.2.1/armv6-m/crtbegin.o
                0x200009bc                PROVIDE (__init_array_end, .)
                0x200009bc                . = ALIGN (0x4)
                [!provide]                PROVIDE (__fini_array_start, .)
 *(SORT(.fini_array.*))
 *(.fini_array)
 .fini_array    0x200009bc        0x4 c:/program files (x86)/gnu tools arm embedded/5.2 2015q4/bin/../lib/gcc/arm-none-eabi/5.2.1/armv6-m/crtbegin.o
                [!provide]                PROVIDE (__fini_array_end, .)
 *(.jcr*)
 .jcr           0x200009c0        0x0 c:/program files (x86)/gnu tools arm embedded/5.2 2015q4/bin/../lib/gcc/arm-none-eabi/5.2.1/armv6-m/crtbegin.o
 .jcr           0x200009c0        0x4 c:/program files (x86)/gnu tools arm embedded/5.2 2015q4/bin/../lib/gcc/arm-none-eabi/5.2.1/armv6-m/crtend.o
                0x200009c4                . = ALIGN (0x4)
                0x200009c4                __data_end__ = .

.tm_clone_table
                0x200009c4        0x0 load address 0x00002054
 .tm_clone_table
                0x200009c4        0x0 c:/program files (x86)/gnu tools arm embedded/5.2 2015q4/bin/../lib/gcc/arm-none-eabi/5.2.1/armv6-m/crtbegin.o
 .tm_clone_table
                0x200009c4        0x0 c:/program files (x86)/gnu tools arm embedded/5.2 2015q4/bin/../lib/gcc/arm-none-eabi/5.2.1/armv6-m/crtend.o

.igot.plt       0x200009c4        0x0 load address 0x00002054
 .igot.plt      0x200009c4        0x0 c:/program files (x86)/gnu tools arm embedded/5.2 2015q4/bin/../lib/gcc/arm-none-eabi/5.2.1/armv6-m/crtbegin.o

.bss            0x20000a00      0x724 load address 0x00002100
                0x20000a00                . = ALIGN (0x4)
                0x20000a00                __bss_start__ = .
 *(.bss*)
 .bss           0x20000a00       0x1c c:/program files (x86)/gnu tools arm embedded/5.2 2015q4/bin/../lib/gcc/arm-none-eabi/5.2.1/armv6-m/crtbegin.o
 .bss.decryptionKey
                0x20000a1c       0x10 ./src/aes.o
 .bss.prevCipher
                0x20000a2c       0x10 ./src/aes.o
 .bss.pageBuffer
                0x20000a3c      0x400 ./src/flash.o
 .bss.cmuStatus
                0x20000e3c        0x4 ./emlib/em_emu.o
 .bss.INT_LockCnt
                0x20000e40        0x4 ./emlib/em_int.o
                0x20000e40                INT_LockCnt
 *(COMMON)
 *fill*         0x20000e44       0xbc 
 COMMON         0x20000f00       0x10 ./src/flash.o
                0x20000f00                descr
 COMMON         0x20000f10      0x210 ./src/xmodem.o
                0x20000f10                rawPacket
                0x20001020                rawBuffer
 COMMON         0x20001120        0x4 ./CMSIS/efm32hg/system_efm32hg.o
                0x20001120                SystemCoreClock
                0x20001124                . = ALIGN (0x4)
                0x20001124                __bss_end__ = .

.heap           0x20001128      0x400
                0x20001128                __HeapBase = .
                0x20001128                __end__ = .
                0x20001128                end = __end__
                0x20001128                _end = __end__
 *(.heap*)
 .heap          0x20001128      0x400 ./CMSIS/efm32hg/startup_efm32hg.o
                0x20001528                __HeapLimit = .

.stack_dummy    0x20001128      0x400
 *(.stack*)
 .stack         0x20001128      0x400 ./CMSIS/efm32hg/startup_efm32hg.o
                0x20002000                __StackTop = (ORIGIN (RAM) + LENGTH (RAM))
                0x20001c00                __StackLimit = (__StackTop - SIZEOF (.stack_dummy))
                0x20002000                PROVIDE (__stack, __StackTop)
                0x00000001                ASSERT ((__StackLimit >= __HeapLimit), region RAM overflowed with stack)
                0x00000001                ASSERT ((LENGTH (FLASH) >= (__etext + SIZEOF (.data))), FLASH memory overflowed !)
OUTPUT(SLSTK3400A_bootloader.axf elf32-littlearm)

.ARM.attributes
                0x00000000       0x28
 .ARM.attributes
                0x00000000       0x1e c:/program files (x86)/gnu tools arm embedded/5.2 2015q4/bin/../lib/gcc/arm-none-eabi/5.2.1/armv6-m/crti.o
 .ARM.attributes
                0x0000001e       0x2c c:/program files (x86)/gnu tools arm embedded/5.2 2015q4/bin/../lib/gcc/arm-none-eabi/5.2.1/armv6-m/crtbegin.o
 .ARM.attributes
                0x0000004a       0x1b c:/program files (x86)/gnu tools arm embedded/5.2 2015q4/bin/../lib/gcc/arm-none-eabi/5.2.1/../../../../arm-none-eabi/lib/armv6-m/crt0.o
 .ARM.attributes
                0x00000065       0x32 ./src/aes.o
 .ARM.attributes
                0x00000097       0x32 ./src/aes_keys.o
 .ARM.attributes
                0x000000c9       0x32 ./src/boot.o
 .ARM.attributes
                0x000000fb       0x32 ./src/bootloader.o
 .ARM.attributes
                0x0000012d       0x32 ./src/crc.o
 .ARM.attributes
                0x0000015f       0x32 ./src/debuglock.o
 .ARM.attributes
                0x00000191       0x32 ./src/flash.o
 .ARM.attributes
                0x000001c3       0x32 ./src/uart.o
 .ARM.attributes
                0x000001f5       0x32 ./src/verify.o
 .ARM.attributes
                0x00000227       0x32 ./src/xmodem.o
 .ARM.attributes
                0x00000259       0x32 ./emlib/em_cmu.o
 .ARM.attributes
                0x0000028b       0x32 ./emlib/em_emu.o
 .ARM.attributes
                0x000002bd       0x32 ./emlib/em_gpio.o
 .ARM.attributes
                0x000002ef       0x32 ./emlib/em_int.o
 .ARM.attributes
                0x00000321       0x32 ./emlib/em_usart.o
 .ARM.attributes
                0x00000353       0x1b ./CMSIS/efm32hg/startup_efm32hg.o
 .ARM.attributes
                0x0000036e       0x32 ./CMSIS/efm32hg/system_efm32hg.o
 .ARM.attributes
                0x000003a0       0x1e c:/program files (x86)/gnu tools arm embedded/5.2 2015q4/bin/../lib/gcc/arm-none-eabi/5.2.1/armv6-m\libgcc.a(_udivsi3.o)
 .ARM.attributes
                0x000003be       0x1e c:/program files (x86)/gnu tools arm embedded/5.2 2015q4/bin/../lib/gcc/arm-none-eabi/5.2.1/armv6-m\libgcc.a(_dvmd_tls.o)
 .ARM.attributes
                0x000003dc       0x2c c:/program files (x86)/gnu tools arm embedded/5.2 2015q4/bin/../lib/gcc/arm-none-eabi/5.2.1/../../../../arm-none-eabi/lib/armv6-m\libc_nano.a(lib_a-exit.o)
 .ARM.attributes
                0x00000408       0x2c c:/program files (x86)/gnu tools arm embedded/5.2 2015q4/bin/../lib/gcc/arm-none-eabi/5.2.1/../../../../arm-none-eabi/lib/armv6-m\libc_nano.a(lib_a-impure.o)
 .ARM.attributes
                0x00000434       0x2c c:/program files (x86)/gnu tools arm embedded/5.2 2015q4/bin/../lib/gcc/arm-none-eabi/5.2.1/../../../../arm-none-eabi/lib/armv6-m\libc_nano.a(lib_a-init.o)
 .ARM.attributes
                0x00000460       0x2c c:/program files (x86)/gnu tools arm embedded/5.2 2015q4/bin/../lib/gcc/arm-none-eabi/5.2.1/../../../../arm-none-eabi/lib/armv6-m\libc_nano.a(lib_a-memcpy-stub.o)
 .ARM.attributes
                0x0000048c       0x2c c:/program files (x86)/gnu tools arm embedded/5.2 2015q4/bin/../lib/gcc/arm-none-eabi/5.2.1/../../../../arm-none-eabi/lib/armv6-m\libc_nano.a(lib_a-memset.o)
 .ARM.attributes
                0x000004b8       0x2c c:/program files (x86)/gnu tools arm embedded/5.2 2015q4/bin/../lib/gcc/arm-none-eabi/5.2.1/../../../../arm-none-eabi/lib/armv6-m\libnosys.a(_exit.o)
 .ARM.attributes
                0x000004e4       0x2c c:/program files (x86)/gnu tools arm embedded/5.2 2015q4/bin/../lib/gcc/arm-none-eabi/5.2.1/armv6-m/crtend.o
 .ARM.attributes
                0x00000510       0x1e c:/program files (x86)/gnu tools arm embedded/5.2 2015q4/bin/../lib/gcc/arm-none-eabi/5.2.1/armv6-m/crtn.o

.comment        0x00000000       0x6e
 .comment       0x00000000       0x6e ./src/aes.o
                                 0x6f (size before relaxing)
 .comment       0x0000006e       0x6f ./src/aes_keys.o
 .comment       0x0000006e       0x6f ./src/boot.o
 .comment       0x0000006e       0x6f ./src/bootloader.o
 .comment       0x0000006e       0x6f ./src/crc.o
 .comment       0x0000006e       0x6f ./src/debuglock.o
 .comment       0x0000006e       0x6f ./src/flash.o
 .comment       0x0000006e       0x6f ./src/uart.o
 .comment       0x0000006e       0x6f ./src/verify.o
 .comment       0x0000006e       0x6f ./src/xmodem.o
 .comment       0x0000006e       0x6f ./emlib/em_cmu.o
 .comment       0x0000006e       0x6f ./emlib/em_emu.o
 .comment       0x0000006e       0x6f ./emlib/em_gpio.o
 .comment       0x0000006e       0x6f ./emlib/em_int.o
 .comment       0x0000006e       0x6f ./emlib/em_usart.o
 .comment       0x0000006e       0x6f ./CMSIS/efm32hg/system_efm32hg.o

.debug_info     0x00000000     0x8de8
 .debug_info    0x00000000      0x8d7 ./src/aes.o
 .debug_info    0x000008d7       0xf5 ./src/aes_keys.o
 .debug_info    0x000009cc      0x413 ./src/boot.o
 .debug_info    0x00000ddf     0x1070 ./src/bootloader.o
 .debug_info    0x00001e4f      0x11e ./src/crc.o
 .debug_info    0x00001f6d      0x3b1 ./src/debuglock.o
 .debug_info    0x0000231e      0x9b8 ./src/flash.o
 .debug_info    0x00002cd6      0x75e ./src/uart.o
 .debug_info    0x00003434      0x817 ./src/verify.o
 .debug_info    0x00003c4b      0x88d ./src/xmodem.o
 .debug_info    0x000044d8     0x20ab ./emlib/em_cmu.o
 .debug_info    0x00006583      0x6b7 ./emlib/em_emu.o
 .debug_info    0x00006c3a      0x7be ./emlib/em_gpio.o
 .debug_info    0x000073f8       0xab ./emlib/em_int.o
 .debug_info    0x000074a3     0x12ef ./emlib/em_usart.o
 .debug_info    0x00008792      0x10e ./CMSIS/efm32hg/startup_efm32hg.o
 .debug_info    0x000088a0      0x548 ./CMSIS/efm32hg/system_efm32hg.o

.debug_abbrev   0x00000000     0x1ef8
 .debug_abbrev  0x00000000      0x25e ./src/aes.o
 .debug_abbrev  0x0000025e       0x56 ./src/aes_keys.o
 .debug_abbrev  0x000002b4      0x172 ./src/boot.o
 .debug_abbrev  0x00000426      0x3a6 ./src/bootloader.o
 .debug_abbrev  0x000007cc       0x9a ./src/crc.o
 .debug_abbrev  0x00000866      0x186 ./src/debuglock.o
 .debug_abbrev  0x000009ec      0x1fb ./src/flash.o
 .debug_abbrev  0x00000be7      0x1ab ./src/uart.o
 .debug_abbrev  0x00000d92      0x1ff ./src/verify.o
 .debug_abbrev  0x00000f91      0x1d9 ./src/xmodem.o
 .debug_abbrev  0x0000116a      0x42d ./emlib/em_cmu.o
 .debug_abbrev  0x00001597      0x207 ./emlib/em_emu.o
 .debug_abbrev  0x0000179e      0x29d ./emlib/em_gpio.o
 .debug_abbrev  0x00001a3b       0x42 ./emlib/em_int.o
 .debug_abbrev  0x00001a7d      0x2ee ./emlib/em_usart.o
 .debug_abbrev  0x00001d6b       0x14 ./CMSIS/efm32hg/startup_efm32hg.o
 .debug_abbrev  0x00001d7f      0x179 ./CMSIS/efm32hg/system_efm32hg.o

.debug_loc      0x00000000     0x5945
 .debug_loc     0x00000000      0x80c ./src/aes.o
 .debug_loc     0x0000080c       0x82 ./src/boot.o
 .debug_loc     0x0000088e      0x2e7 ./src/bootloader.o
 .debug_loc     0x00000b75       0xf8 ./src/crc.o
 .debug_loc     0x00000c6d      0x2ff ./src/debuglock.o
 .debug_loc     0x00000f6c      0x2fe ./src/flash.o
 .debug_loc     0x0000126a       0x7d ./src/uart.o
 .debug_loc     0x000012e7      0x833 ./src/verify.o
 .debug_loc     0x00001b1a      0x28c ./src/xmodem.o
 .debug_loc     0x00001da6     0x2057 ./emlib/em_cmu.o
 .debug_loc     0x00003dfd      0x242 ./emlib/em_emu.o
 .debug_loc     0x0000403f      0x60d ./emlib/em_gpio.o
 .debug_loc     0x0000464c      0xe44 ./emlib/em_usart.o
 .debug_loc     0x00005490      0x4b5 ./CMSIS/efm32hg/system_efm32hg.o

.debug_aranges  0x00000000      0x500
 .debug_aranges
                0x00000000       0x40 ./src/aes.o
 .debug_aranges
                0x00000040       0x18 ./src/aes_keys.o
 .debug_aranges
                0x00000058       0x28 ./src/boot.o
 .debug_aranges
                0x00000080       0x58 ./src/bootloader.o
 .debug_aranges
                0x000000d8       0x20 ./src/crc.o
 .debug_aranges
                0x000000f8       0x30 ./src/debuglock.o
 .debug_aranges
                0x00000128       0x40 ./src/flash.o
 .debug_aranges
                0x00000168       0x38 ./src/uart.o
 .debug_aranges
                0x000001a0       0x58 ./src/verify.o
 .debug_aranges
                0x000001f8       0x28 ./src/xmodem.o
 .debug_aranges
                0x00000220       0xf0 ./emlib/em_cmu.o
 .debug_aranges
                0x00000310       0x50 ./emlib/em_emu.o
 .debug_aranges
                0x00000360       0x48 ./emlib/em_gpio.o
 .debug_aranges
                0x000003a8       0x18 ./emlib/em_int.o
 .debug_aranges
                0x000003c0       0xb8 ./emlib/em_usart.o
 .debug_aranges
                0x00000478       0x20 ./CMSIS/efm32hg/startup_efm32hg.o
 .debug_aranges
                0x00000498       0x68 ./CMSIS/efm32hg/system_efm32hg.o

.debug_ranges   0x00000000      0xde0
 .debug_ranges  0x00000000      0x210 ./src/aes.o
 .debug_ranges  0x00000210       0x18 ./src/boot.o
 .debug_ranges  0x00000228       0xc8 ./src/bootloader.o
 .debug_ranges  0x000002f0       0x10 ./src/crc.o
 .debug_ranges  0x00000300       0x38 ./src/debuglock.o
 .debug_ranges  0x00000338       0x78 ./src/flash.o
 .debug_ranges  0x000003b0       0x40 ./src/uart.o
 .debug_ranges  0x000003f0      0x108 ./src/verify.o
 .debug_ranges  0x000004f8       0x18 ./src/xmodem.o
 .debug_ranges  0x00000510      0x490 ./emlib/em_cmu.o
 .debug_ranges  0x000009a0       0x70 ./emlib/em_emu.o
 .debug_ranges  0x00000a10       0xb8 ./emlib/em_gpio.o
 .debug_ranges  0x00000ac8      0x238 ./emlib/em_usart.o
 .debug_ranges  0x00000d00       0xe0 ./CMSIS/efm32hg/system_efm32hg.o

.debug_line     0x00000000     0x3663
 .debug_line    0x00000000      0x429 ./src/aes.o
 .debug_line    0x00000429       0xfd ./src/aes_keys.o
 .debug_line    0x00000526      0x1ac ./src/boot.o
 .debug_line    0x000006d2      0x48c ./src/bootloader.o
 .debug_line    0x00000b5e      0x142 ./src/crc.o
 .debug_line    0x00000ca0      0x25d ./src/debuglock.o
 .debug_line    0x00000efd      0x2e7 ./src/flash.o
 .debug_line    0x000011e4      0x203 ./src/uart.o
 .debug_line    0x000013e7      0x306 ./src/verify.o
 .debug_line    0x000016ed      0x29c ./src/xmodem.o
 .debug_line    0x00001989      0xad5 ./emlib/em_cmu.o
 .debug_line    0x0000245e      0x3f1 ./emlib/em_emu.o
 .debug_line    0x0000284f      0x2f1 ./emlib/em_gpio.o
 .debug_line    0x00002b40      0x120 ./emlib/em_int.o
 .debug_line    0x00002c60      0x649 ./emlib/em_usart.o
 .debug_line    0x000032a9       0xa7 ./CMSIS/efm32hg/startup_efm32hg.o
 .debug_line    0x00003350      0x313 ./CMSIS/efm32hg/system_efm32hg.o

.debug_str      0x00000000     0x24fb
 .debug_str     0x00000000      0x3fa ./src/aes.o
                                0x499 (size before relaxing)
 .debug_str     0x000003fa       0x29 ./src/aes_keys.o
                                0x240 (size before relaxing)
 .debug_str     0x00000423      0x3c0 ./src/boot.o
                                0x5d0 (size before relaxing)
 .debug_str     0x000007e3      0x4bf ./src/bootloader.o
                                0xab1 (size before relaxing)
 .debug_str     0x00000ca2       0x2c ./src/crc.o
                                0x233 (size before relaxing)
 .debug_str     0x00000cce       0x6c ./src/debuglock.o
                                0x345 (size before relaxing)
 .debug_str     0x00000d3a      0x1f6 ./src/flash.o
                                0x5b3 (size before relaxing)
 .debug_str     0x00000f30      0x373 ./src/uart.o
                                0x939 (size before relaxing)
 .debug_str     0x000012a3       0x67 ./src/verify.o
                                0x4d3 (size before relaxing)
 .debug_str     0x0000130a       0xd6 ./src/xmodem.o
                                0x553 (size before relaxing)
 .debug_str     0x000013e0      0x849 ./emlib/em_cmu.o
                                0xd73 (size before relaxing)
 .debug_str     0x00001c29      0x12e ./emlib/em_emu.o
                                0x45c (size before relaxing)
 .debug_str     0x00001d57      0x156 ./emlib/em_gpio.o
                                0x5ac (size before relaxing)
 .debug_str     0x00001ead       0x35 ./emlib/em_int.o
                                0x1b6 (size before relaxing)
 .debug_str     0x00001ee2      0x550 ./emlib/em_usart.o
                                0xc4e (size before relaxing)
 .debug_str     0x00002432       0xc9 ./CMSIS/efm32hg/system_efm32hg.o
                                0x405 (size before relaxing)

.debug_frame    0x00000000      0xbb8
 .debug_frame   0x00000000       0x94 ./src/aes.o
 .debug_frame   0x00000094       0x48 ./src/boot.o
 .debug_frame   0x000000dc       0xec ./src/bootloader.o
 .debug_frame   0x000001c8       0x30 ./src/crc.o
 .debug_frame   0x000001f8       0x68 ./src/debuglock.o
 .debug_frame   0x00000260       0xa0 ./src/flash.o
 .debug_frame   0x00000300       0x64 ./src/uart.o
 .debug_frame   0x00000364       0xf0 ./src/verify.o
 .debug_frame   0x00000454       0x54 ./src/xmodem.o
 .debug_frame   0x000004a8      0x24c ./emlib/em_cmu.o
 .debug_frame   0x000006f4       0xac ./emlib/em_emu.o
 .debug_frame   0x000007a0       0xa0 ./emlib/em_gpio.o
 .debug_frame   0x00000840      0x1cc ./emlib/em_usart.o
 .debug_frame   0x00000a0c       0xd0 ./CMSIS/efm32hg/system_efm32hg.o
 .debug_frame   0x00000adc       0x20 c:/program files (x86)/gnu tools arm embedded/5.2 2015q4/bin/../lib/gcc/arm-none-eabi/5.2.1/armv6-m\libgcc.a(_udivsi3.o)
 .debug_frame   0x00000afc       0x28 c:/program files (x86)/gnu tools arm embedded/5.2 2015q4/bin/../lib/gcc/arm-none-eabi/5.2.1/../../../../arm-none-eabi/lib/armv6-m\libc_nano.a(lib_a-exit.o)
 .debug_frame   0x00000b24       0x2c c:/program files (x86)/gnu tools arm embedded/5.2 2015q4/bin/../lib/gcc/arm-none-eabi/5.2.1/../../../../arm-none-eabi/lib/armv6-m\libc_nano.a(lib_a-init.o)
 .debug_frame   0x00000b50       0x28 c:/program files (x86)/gnu tools arm embedded/5.2 2015q4/bin/../lib/gcc/arm-none-eabi/5.2.1/../../../../arm-none-eabi/lib/armv6-m\libc_nano.a(lib_a-memcpy-stub.o)
 .debug_frame   0x00000b78       0x20 c:/program files (x86)/gnu tools arm embedded/5.2 2015q4/bin/../lib/gcc/arm-none-eabi/5.2.1/../../../../arm-none-eabi/lib/armv6-m\libc_nano.a(lib_a-memset.o)
 .debug_frame   0x00000b98       0x20 c:/program files (x86)/gnu tools arm embedded/5.2 2015q4/bin/../lib/gcc/arm-none-eabi/5.2.1/../../../../arm-none-eabi/lib/armv6-m\libnosys.a(_exit.o)
